:020000040000FA
:0608000068EF2DF012006C
:020806001200DE
:06080800E4EF05F0120010
:02080E00FEFFEB
:060818001CEF04F01200C9
:02081E000200D6
:100820000E080000F7010000020000002F5B00002E
:080830009901000052000000D4
:08083800D8CFE4FFE0CFE4FF9C
:10084000E46EDACFE4FFE2CFDAFFE9CFE4FFEACFEC
:10085000E4FFF6CFE4FFF7CFE4FFF5CFE4FFF3CFFB
:10086000E4FFF4CFE4FFFACFE4FF00EE1AF0140E39
:10087000E80403E3EECFE4FFFBD700EE2EF0100E0A
:10088000E80403E3EECFE4FFFBD7E652DBEC18F01D
:100890009EA200D19E92030E3E6E0E50EA6A510F48
:1008A000E96E010EEA22EF503E5C30E10E50E96E37
:1008B000EA6AD890E936EA36690EE926010EEA229C
:1008C000EECF3EF0EFCF3FF03FC03EF03F6A3E50EC
:1008D000D76E0E50E96EEA6AD890E936EA36690EAC
:1008E000E926010EEA22EECF3EF0EFCF3FF03E5078
:1008F000D66EF28AF294D58E0E50EA6A510FE96EE6
:10090000010EEA22040EEF6E0E50106E020E3E6EC5
:100910000F50EA6A510FE96E010EEA22EF503E5C79
:1009200049E10F50E96EEA6AD890E936EA36690E75
:10093000E926010EEA22EE50ED1009E10F50EA6AB5
:10094000510FE96E010EEA22010EEF6E33D0080E50
:100950000F5C0CE2070E0F143E6E010E3E5204E0D7
:10096000E846FE0B3E06FCE189121AD0100E0F5C21
:100970000CE2070E0F143E6E010E3E5204E0E846F4
:10098000FE0B3E06FCE18A120BD0070E0F143E6EE2
:10099000010E3E5204E0E846FE0B3E06FCE18B12DF
:1009A0000F50EA6A510FE96E010EEA22030EEF6E54
:1009B0000F500E6E0F2A060E0F5C02E1080E04D0D7
:1009C000130E0F5C03E1160E0F6E04D0180E0F5CB1
:1009D00001E10F6A000ED8800254000E03542EE28B
:1009E000112A000E12220250115C0350125826E305
:1009F000116A126A030E065C1FE20450EA6A480F8D
:100A0000E96E010EEA2280CFEFFF0450EA6A4B0F35
:100A1000E96E010EEA2281CFEFFF0450EA6A4E0F21
:100A2000E96E010EEA2282CFEFFF042A030E045C76
:100A300001E3046A062A02D0026A036A000ED88023
:100A40000754000E085419E20C50000816E2132A4D
:100A5000000E14220750135C085014580EE3136A5A
:100A6000146A030E0B5C07E2092A030E095C01E31A
:100A7000096A0B2A02D0076A086A0C5000080AE2C9
:100A8000156A1550040DF328C26E9E9C9F9C9D8C88
:100A9000C280C2829EAC2BD09E9CC450436E426AE0
:100AA000C35000014210406E43C041F01550060D86
:100AB000F3CF3EF0F4CF3FF0000E3E26010E3F2272
:100AC0000950020D3E50F324E96E3F50F420EA6EC7
:100AD00040C0EEFF41C0EDFF152A0C50155C02E34B
:100AE0009D9C05D01550040DF328C26EC282F2A45D
:100AF00042D0D59EF294F29A040E3E6E1050EA6AED
:100B0000510FE96E010EEA22EF503E5C34E1080E0F
:100B1000105C0DE2070E10143E6E010E3E5204E012
:100B2000E846FE0B3E06FCE1E81C89161CD0100EC0
:100B3000105C0DE2070E10143E6E010E3E5204E0F2
:100B4000E846FE0B3E06FCE1E81C8A160CD0070EB8
:100B500010143E6E010E3E5204E0E846FE0B3E06C7
:100B6000FCE1E81C8B161050EA6A510FE96E010E89
:100B7000EA22020EEF6EE55200EE3DF0100EE804A0
:100B800003E3E5CFEDFFFBD700EE2DF0140EE804F4
:100B900003E3E5CFEDFFFBD7E5CFFAFFE5CFF4FFA9
:100BA000E5CFF3FFE5CFF5FFE5CFF7FFE5CFF6FFA4
:100BB000E5CFEAFFE5CFE9FFE5CFDAFFE550E5CF86
:100BC000E0FFE5CFD8FF1000DACFE4FFE652A1A2A4
:100BD00015D01650B36E1750B26E192A1850195C02
:100BE0000CE301019951891A9A518A1A9B518B1A67
:100BF0009C518C1A9D518D1A196AA192E552E5CF2C
:100C0000DAFF1100D9CFE6FFE1CFD9FF020EE126CE
:100C1000896A92680F0EC16EC2900C6A070EB46E9C
:100C20008A6A93688B6A94688C6A95688D6A9668FC
:100C30008B908B929490949294840201010ECD6FCC
:100C40000101F769F8690A6A096A0B6A056A046AA8
:100C5000066A026A036A076A086A116A126A136AF4
:100C6000146A156ACA82CA80CA9CCA9ACA88CA9675
:100C7000FA0ECB6EDF6ADFCF2EF00C0EE76E2E1869
:100C8000E8AE02D0E73402D0E7502E5C36E2010E27
:100C9000DB6ADBCF2EF0030EE76E2E18E8AE02D033
:100CA000E73402D0E7502E5C26E2DFCF2EF02F6A29
:100CB0002EBE2F68060E2F02F3CF2FF02E02F3CF99
:100CC0002EF0F4502F26000E2E26010E2F22010E9C
:100CD000DBCF30F0316A30BE3168D89030363136F3
:100CE0002E503024E96E2F503120EA6EEE6AED6A04
:100CF000010EDB2ACED7DF2ABED70201C76BC86B35
:100D0000C56BC66BC96BCA6BCB6BCC6B0E6A0F6ABB
:100D1000106ADF6ADFCF2EF0180EE76E2E18E8AEED
:100D200002D0E73402D0E7502E5C1BE2DFCFE9FFB0
:100D3000EA6AE9BEEA68D890E936EA36690EE92639
:100D4000010EEA22EE6AED6ADFCFE9FFEA6AE9BE48
:100D5000EA68510EE926010EEA22010EEF6EDF2A43
:100D6000D9D7D586D59AD59CF294F29AF194D08EA3
:100D7000CA949D829F92F28EF28CCA84020EE15C2C
:100D800002E2E16AE552E16EE552E7CFD9FF1200D7
:100D9000D9CFE6FFE1CFD9FF050EE126020EDB6ACF
:100DA000030EDB6A040EDB6ADFEC17F00650000866
:100DB00009E2F6EC0CF0052A030E055C01E1056A78
:100DC0000606F4D70B50000809E226EC0DF00A2ABB
:100DD000030E0A5C01E10A6A0B06F4D7200E00013B
:100DE000E76E6019E8AE02D0E73402D0E750605DEC
:100DF00001E2EAD16D50020B01E0E6D1400EE66E51
:100E0000400EE66E020EE66EEAEC27F0E552E55281
:100E1000E552E76E030EE7CFDBFFDB50000801E38E
:100E200069D1040EDB6A030EDB50F36E040EDBCFD8
:100E3000F4FFF350F45C01E35DD1040EDB50EA6A89
:100E4000400FE96E020EEA22EFCFDFFF0101E6510B
:100E500010E0E75100080DE20201C751EA6A000FF5
:100E6000E96E030EEA22DFCFEFFFC72B0101E70790
:100E700031D1E25144E10D0E2E6EDF502E5C05E0C3
:100E80000A0E2F6EDF502F5C3AE1010EE26F020175
:100E9000C751EA6A000FE96E030EEA220D0EEF6EEB
:100EA000C72B010EDB6AC751F36E010EDBCFF4FFD7
:100EB000F350F45C1CE2010EDBCFE9FFEA6AE9BE05
:100EC000EA68000EE926030EEA22EF50E66E010EF4
:100ED000DBCFE9FFEA6AE9BEEA689E0EE926010E69
:100EE000EA22E552E750EF6E010EDB2ADCD7F4D997
:100EF0000101E66BE76B0201C76BC86BEBD01B0E01
:100F0000DF5C09E1DE5107E1010EDE6F1B0EDF6FD2
:100F1000E06BE16BDFD0DE050BE15B0EDF5C08E12F
:100F20001B0EDF5D05E1E05103E15B0EE06FD2D007
:100F3000DE0566E1410EDF5C63E11B0EDF5D60E113
:100F40005B0EE05D5DE1DF6BE06BE16BDE6B010E84
:100F5000DB6ADBCFE9FFEA6AE9BEEA68000EE92650
:100F6000030EEA22EF500D081CE0010EDBCFE9FF73
:100F7000EA6AE9BEEA689E0EE926010EEA22EF500F
:100F8000E66E010EDBCFE9FFEA6AE9BEEA68000E11
:100F9000E926030EEA22E552E750EF6E010EDB2A46
:100FA000D8D7010EDBCFC7F20201C751EA6A000FA2
:100FB000E96E030EEA22EF6A710E2E6E540E2F6E4A
:100FC000306A2EC0E6FFE66E30C0E6FFF6EC2BF08E
:100FD000E552E552E552000EE66E030EE66E6E0E29
:100FE0002E6E540E2F6E306A2EC0E6FFE66E30C0B5
:100FF000E6FFF6EC2BF0316E050EE15E31506AD063
:10100000080EDF5C1CE10201C751000818E2C707A7
:10101000C751EA6A000FE96E030EEA22EF6A6B0E0F
:101020002E6E540E2F6E306A2EC0E6FFE66E30C074
:10103000E6FFF6EC2BF0E552E552E5524BD00D0EF3
:10104000DF5C48E00A0EDF5C45E0200EDF5C42E337
:101050000101DF6BE06BE16BDE6B0201C751EA6AF5
:10106000000FE96E030EEA22DFCFEFFF0101E26B12
:101070000201C72B030EC75D0AE1420E0301005DAA
:1010800006E1530E015D03E10101010EE66F01016E
:10109000E65120E0E7511EE1050E0201C75D09E1BE
:1010A0002C0E0301045D05E1300E035D0101E76FC5
:1010B00011D0060E0201C75D0DE12C0E0301055D86
:1010C00009E1300E035D0A0DF3CFE7F1300E045D48
:1010D0000101E7270201C7512E6E2F6A000E2E185C
:1010E00006E1010E2F1803E10D86C76BC86B040ED5
:1010F000DB2A99D60D5067E00DA00FD0650E2E6E3D
:10110000540E2F6E306A2EC0E6FFE66E30C0E6FF4A
:10111000F6EC2BF0E552E552E5520DA40FD0490E46
:101120002E6E540E2F6E306A2EC0E6FFE66E30C073
:10113000E6FFF6EC2BF0E552E552E5520DA60FD096
:101140002D0E2E6E540E2F6E306A2EC0E6FFE66E08
:1011500030C0E6FFF6EC2BF0E552E552E5520DA863
:101160000FD00E0E2E6E540E2F6E306A2EC0E6FF7C
:10117000E66E30C0E6FFF6EC2BF0E552E552E552A4
:101180000DAC0FD0ED0E2E6E530E2F6E306A2EC0AA
:10119000E6FFE66E30C0E6FFF6EC2BF0E552E552D6
:1011A000E5520DAE0FD0D40E2E6E530E2F6E306A58
:1011B0002EC0E6FFE66E30C0E6FFF6EC2BF0E552FF
:1011C000E552E5520D6A3FD8050EE15C02E2E16AA4
:1011D000E552E16EE552E7CFD9FF1200D9CFE6FF25
:1011E000E1CFD9FFE652C5C2DFFFDF2A400E2E6EE7
:1011F000DF502E5C01E1DF6A0201C651DF5C01E1D4
:1012000022D80201C551EA6A000FE96E020EEA22F5
:10121000FE0EDBCFEFFFC52B400EC55D01E1C56BB8
:10122000C651C55D01E10D84FE0EDBCF2EF02F6AA5
:101230002EBE2F682EC0F3FF2FC0F4FFE552E552FB
:10124000E7CFD9FF1200D9CFE6FFE1CFD9FFE652B1
:101250000201C551C65D3BE00201D05103E0E8EC5C
:1012600028F0FAD70201C651D880C55517E2C651F9
:10127000C55DDF6EDFCFE6FFC6512F6A000F2E6E11
:10128000020E2F222EC0E6FF2FC0E6FF4AEC28F008
:10129000E552E552E552C5C2C6F217D0400ED880DD
:1012A000C655DF6EDFCFE6FFC6512F6A000F2E6EE8
:1012B000020E2F222EC0E6FF2FC0E6FF4AEC28F0D8
:1012C000E552E552E5520201C66BE8EC28F0E55222
:1012D000E552E7CFD9FF1200D9CFE6FFE1CFD9FF22
:1012E000040EE126DE6ADD6A020EDB6A030EDB6AAB
:1012F0000201C851EA6A000FE96E030EEA22EF50BC
:10130000E66EE66AFDEC2CF0E552E552020EF3CFF4
:10131000DBFF0201C82BC8512E6E2F6A000E2E185B
:1013200004E1010E2F1801E1C86B020EDB50DE6EE6
:10133000DD6AC851EA6A000FE96E030EEA22EF5037
:101340002C0836E0C851EA6A000FE96E030EEA2263
:10135000EF500D082DE0C851EA6A000FE96E030E48
:10136000EA22EF50E66EE66AFDEC2CF0E552E5521B
:10137000030EF3CFDBFF0201C82BC8512E6E2F6A7C
:10138000000E2E1804E1010E2F1801E1C86B020EA9
:10139000DBCF30F030C031F0306A030EDB5000019B
:1013A00030242E6E000E31202F6E2EC0DEFFDD6E3B
:1013B000000EDFCF22F0010EDBCF23F0460E221805
:1013C00001E1235001E1FED0490E221802E1430E53
:1013D000231801E1F4D0490E221802E1520E23181D
:1013E00001E1EAD0490E221802E1530E231801E16F
:1013F000E0D0530E221802E1430E231801E1D6D0AB
:10140000530E221802E1520E231801E1CCD0530EE4
:10141000221802E1530E231801E1C2D0530E221804
:1014200002E1420E231801E1B8D0430E221802E176
:10143000420E231801E1AED0430E221802E1520EF3
:10144000231801E1A4D04F0E221802E1420E231806
:1014500001E19AD0570E221802E14D0E231801E146
:1014600091D0520E221802E14D0E231801E188D0CE
:10147000440E221802E1500E231801E17FD04F0ED6
:10148000221802E1500E231876E0490E221802E1DC
:10149000500E23186DE0580E221802E1540E231846
:1014A00064E0540E221801E123505DE0410E221841
:1014B00001E1235056E0560E221801E123504FE07F
:1014C000490E221801E1235048E04F0E221801E195
:1014D000235041E0550E221802E1430E231839E053
:1014E000580E221802E1430E231830E0430E221852
:1014F00001E1235029E0520E221801E1235022E09D
:10150000580E221802E1520E231819E0030EDB5088
:101510005CE1020EDBCFE6FFE66ADBCFE6FFE66AC0
:10152000B10E2E6E530E2F6E306A2EC0E6FFE66EA1
:1015300030C0E6FFF6EC2BF0316E070E64D077EC8E
:1015400010F063D098D861D02DD95FD079EC10F02D
:101550005CD095D85AD0C1D958D048DA56D066DA7E
:1015600054D074DA52D0D3D850D075EC10F04DD09E
:10157000E9EC0EF04AD08EEC0FF047D044DB45D0BA
:1015800000DB43D0C0DA41D09BEC11F03ED07BECC5
:1015900010F03BD02EEC11F038D0F4EC12F035D036
:1015A000C3EC13F032D0C5EC13F02FD0C7EC13F01E
:1015B0002CD0C9EC13F029D0CBEC13F026D0CDEC15
:1015C00013F023D0CFEC13F020D0030EDBCFE6FFD7
:1015D000E66A020EDBCFE6FFE66A030EDBCFE6FF2C
:1015E000E66A020EDBCFE6FFE66A890E2E6E530E28
:1015F0002F6E306A2EC0E6FFE66E30C0E6FFF6ECD6
:101600002BF0316E0B0EE15E31500201C851EA6AD7
:10161000000FE96E030EEA22EF500D080DE00D50A9
:101620000BE1520E2E6E2F6ADF502E1803E1DE52B0
:10163000DD502F1801E00D8EC7C2C8F2040EE15C28
:1016400002E2E16AE552E16EE552E7CFD9FF12000E
:101650000201CD510FE08E0E2E6E5A0E2F6E306AA3
:101660002EC0E6FFE66E30C0E6FFF6EC2BF0E5524A
:10167000E552E552120002EC06F028EF0BF0D9CF4C
:10168000E6FFE1CFD9FF030EE126E66AD9CFE6FFF8
:10169000DACFE6FF010EE66E74EC15F0E552E55286
:1016A000E552E552E66AD950010FE66E000EDA20E7
:1016B000E66E020EE66E74EC15F0E552E552E55268
:1016C000E5520D501AE1DF0417E1D950010FE96E20
:1016D000DACFEAFFEE50ED100AE0010E2E6E2F6A0F
:1016E000DB502E1808E1020EDB502F1804E1010E2A
:1016F000DBCFCDF201D00D8CABDF030EE15C02E25B
:10170000E16AE552E16EE552E7CFD9FF1200D9CF89
:10171000E6FFE1CFD9FF030EE126020EDB6AE66A9F
:10172000000EE66E000EE66E030EE66E74EC15F02B
:10173000E552E552E552E552E66AD950020FE66EEF
:10174000000EDA20E66E010EE66E74EC15F0E5523E
:10175000E552E552E5520D501BE1020EDB500CE163
:101760000050011003E1026A036A11D0CA8400C06C
:1017700002F001C003F00BD00050011003E1076A32
:10178000086A05D0CA8400C007F001C008F060DF15
:10179000030EE15C02E2E16AE552E16EE552E7CF59
:1017A000D9FF1200D9CFE6FFE1CFD9FF060EE1261F
:1017B000E66AD9CFE6FFDACFE6FF010EE66E74ECFB
:1017C00015F0E552E552E552E552E66AD950010FAF
:1017D000E66E000EDA20E66E010EE66E74EC15F091
:1017E000E552E552E552E552E66AD950020FE66E3F
:1017F000000EDA20E66E010EE66E74EC15F0E5528E
:10180000E552E552E552E66AD950040FE66E000E45
:10181000DA20E66E010EE66E74EC15F0E552E55244
:10182000E552E552E66AD950050FE66E000EDA2061
:10183000E66E010EE66E74EC15F0E552E552E552E7
:10184000E552E66AD950030FE66E000EDA20E66E26
:10185000010EE66E74EC15F0E552E552E552E552E4
:101860000D5031E1DF50926E010EDB50936E020E8F
:10187000DB50946E040EDB50956E050EDB50966EB9
:10188000030EDB500D0805E20D0EF36E030EF3CFD1
:10189000DBFF030EDB5005E10F0EC16EC2900C6A38
:1018A00011D00C6AC26A030EDBCFE6FF0F0EE552C1
:1018B000D880E754C16EBE0EC06EC280030EDB50EE
:1018C0000C6ECA84C5DE060EE15C02E2E16AE552F6
:1018D000E16EE552E7CFD9FF1200D9CFE6FFE1CFA5
:1018E000D9FF020EE126E66AD9CFE6FFDACFE6FF9E
:1018F000010EE66E74EC15F0E552E552E552E55244
:10190000E76E010EE7CFDBFF0D5066E1010EDB5005
:1019100002E1DF50896E010EE66ED9CFE6FFDACF25
:10192000E6FFE66E74EC15F0E552E552E552E5523D
:10193000E76E010EE7CFDBFF0D504EE1010EDB50ED
:1019400002E1DF508A6E010EE66ED9CFE6FFDACFF4
:10195000E6FFE66E74EC15F0E552E552E552E5520D
:10196000E76E010EE7CFDBFF0D5036E1010EDB50D5
:1019700002E1DF508B6E010EE66ED9CFE6FFDACFC3
:10198000E6FFE66E74EC15F0E552E552E552E552DD
:10199000E76E010EE7CFDBFF0D501EE1010EDB50BD
:1019A00002E1DF508C6E010EE66ED9CFE6FFDACF92
:1019B000E6FFE66E74EC15F0E552E552E552E552AD
:1019C000E76E010EE7CFDBFF0D5006E1010EDB50A5
:1019D00002E1DF508D6E3CDE020EE15C02E2E16A64
:1019E000E552E16EE552E7CFD9FF12008450E66E72
:1019F000E66A8350E66EE66A8250E66EE66A8150D9
:101A0000E66EE66A8050E66EE66A6C0E2E6E530E47
:101A10002F6E306A2EC0E6FFE66E30C0E6FFF6ECB1
:101A20002BF0316E0D0EE15E31501200960E2E6ECF
:101A30005A0E2F6E306A2EC0E6FFE66E30C0E6FF0B
:101A4000F6EC2BF0E552E552E5521200D9CFE6FF55
:101A5000E1CFD9FFE652DF6A6A0E2E6E530E2F6E6B
:101A6000306A2EC0E6FFE66E30C0E6FFF6EC2BF0E3
:101A7000E552E552E552DF6A0C50DF5C30E2DFCF21
:101A80002EF02F6A2EBE2F68060E2F02F3CF2FF0F6
:101A90002E02F3CF2EF0F4502F26000E2E26010E2C
:101AA0002F220A50020D2E50F324E96E2F50F420FD
:101AB000EA6EEECFE6FFEFCFE6FF640E306E530E18
:101AC000316E326A30C0E6FFE66E32C0E6FFF6ECF9
:101AD0002BF0336E050EE15E3350DF2ACDD7930E27
:101AE0002E6E5A0E2F6E306A2EC0E6FFE66E30C0A4
:101AF000E6FFF6EC2BF0E552E552E552E552E552F1
:101B0000E7CFD9FF1200D9CFE6FFE1CFD9FF030E0F
:101B1000E126E66AD9CFE6FFDACFE6FFE66E74EC9F
:101B200015F0E552E552E552E552E66AD950020F4A
:101B3000E66E000EDA20E66E010EE66E74EC15F02D
:101B4000E552E552E552E5520D5011E1DECF2EF09F
:101B5000DDCF2FF0000E2E5C100E2F5807E2DECFE7
:101B6000E9FFDDCFEAFF020EDBCFEFFF71DD030EF1
:101B7000E15C02E2E16AE552E16EE552E7CFD9FFAE
:101B80001200D9CFE6FFE1CFD9FF030EE126E66AC6
:101B9000D9CFE6FFDACFE6FFE66E74EC15F0E5523A
:101BA000E552E552E5520D5024E1DECF2EF0DDCFB7
:101BB0002FF0000E2E5C100E2F5807E2DECFE9FF4B
:101BC000DDCFEAFF020EEFCFDBFF020EDBCFE6FF39
:101BD000E66A5A0E2E6E530E2F6E306A2EC0E6FF46
:101BE000E66E30C0E6FFF6EC2BF0316E050EE15EDE
:101BF0003150030EE15C02E2E16AE552E16EE5522A
:101C0000E7CFD9FF1200D9CFE6FFE1CFD9FF030E0E
:101C1000E126E66AD9CFE6FFDACFE6FF050EE66EEB
:101C200074EC15F0E552E552E552E552E66AD950FA
:101C3000010FE66E000EDA20E66E010EE66E74EC21
:101C400015F0E552E552E552E552E66AD950020F29
:101C5000E66E000EDA20E66E010EE66E74EC15F00C
:101C6000E552E552E552E5520D5001E0A8D0020ED2
:101C7000DB50010801E2A0D0010EDB50070801E2B1
:101C80009BD0410E2E6EDF502E5C1AE1020EDB500F
:101C90000CE1010EF36EDB5004E0D890F336E80659
:101CA000FCE1F350F31C921689D0010EF36EDB5069
:101CB00004E0D890F336E806FCE1F35092127ED0AF
:101CC000420E2E6EDF502E5C1AE1020EDB500CE14C
:101CD000010EF36EDB5004E0D890F336E806FCE129
:101CE000F350F31C93166AD0010EF36EDB5004E040
:101CF000D890F336E806FCE1F35093125FD0430E20
:101D00002E6EDF502E5C1AE1020EDB500CE1010E4C
:101D1000F36EDB5004E0D890F336E806FCE1F350B4
:101D2000F31C94164BD0010EF36EDB5004E0D890F8
:101D3000F336E806FCE1F350941240D0440E2E6EC8
:101D4000DF502E5C1AE1020EDB500CE1010EF36E47
:101D5000DB5004E0D890F336E806FCE1F350F31CC6
:101D600095162CD0010EF36EDB5004E0D890F336BC
:101D7000E806FCE1F350951221D0450E2E6EDF509F
:101D80002E5C1AE1020EDB500CE1010EF36EDB500B
:101D900004E0D890F336E806FCE1F350F31C961605
:101DA0000DD0010EF36EDB5004E0D890F336E80658
:101DB000FCE1F350961202D00D8C01D049DC030EE9
:101DC000E15C02E2E16AE552E16EE552E7CFD9FF5C
:101DD0001200D9CFE6FFE1CFD9FF030EE126020EB4
:101DE000DB6AE66AD9CFE6FFDACFE6FF050EE66EDC
:101DF00074EC15F0E552E552E552E552E66AD95029
:101E0000010FE66E000EDA20E66E010EE66E74EC4F
:101E100015F0E552E552E552E5520D5075E1010E1F
:101E2000DB50070856E3410E2E6EDF502E5C0BE1AF
:101E3000010EF36EDB5004E0D890F336E806FCE1C7
:101E4000F35080143FD0420E2E6EDF502E5C0BE11B
:101E5000010EF36EDB5004E0D890F336E806FCE1A7
:101E6000F35081142FD0430E2E6EDF502E5C0BE109
:101E7000010EF36EDB5004E0D890F336E806FCE187
:101E8000F35082141FD0440E2E6EDF502E5C0BE1F7
:101E9000010EF36EDB5004E0D890F336E806FCE167
:101EA000F35083140FD0450E2E6EDF502E5C11E1DF
:101EB000010EF36EDB5004E0D890F336E806FCE147
:101EC000F3508414E76E020EE7CFDBFFDB5008E02F
:101ED00002D00D8C19D0010EF36E020EF3CFDBFF92
:101EE000020EDBCFE6FFE66A510E2E6E530E2F6E0A
:101EF000306A2EC0E6FFE66E30C0E6FFF6EC2BF04F
:101F0000316E050EE15E3150030EE15C02E2E16AE2
:101F1000E552E16EE552E7CFD9FF1200D9CFE6FFD7
:101F2000E1CFD9FF030EE126E66AD9CFE6FFDACF8B
:101F3000E6FF050EE66E74EC15F0E552E552E5524B
:101F4000E552E66AD950010FE66E000EDA20E66E21
:101F5000010EE66E74EC15F0E552E552E552E552DD
:101F6000E66AD950020FE66E000EDA20E66E010E28
:101F7000E66E74EC15F0E552E552E552E5520D506F
:101F800001E0A9D0020EDB50010801E2A0D0010E51
:101F9000DB50070801E29BD0410E2E6EDF502E5C15
:101FA0001AE1020EDB500CE1010EF36EDB5004E08F
:101FB000D890F336E806FCE1F350F31C891689D07B
:101FC000010EF36EDB5004E0D890F336E806FCE136
:101FD000F35089127ED0420E2E6EDF502E5C1AE135
:101FE000020EDB500CE1010EF36EDB5004E0D890E2
:101FF000F336E806FCE1F350F31C8A166AD0010EB2
:10200000F36EDB5004E0D890F336E806FCE1F350C1
:102010008A125FD0430E2E6EDF502E5C1AE1020E44
:10202000DB500CE1010EF36EDB5004E0D890F33688
:10203000E806FCE1F350F31C8B164BD0010EF36E57
:10204000DB5004E0D890F336E806FCE1F3508B1245
:1020500040D0440E2E6EDF502E5C1AE1020EDB5093
:102060000CE1010EF36EDB5004E0D890F336E80685
:10207000FCE1F350F31C8C162CD0010EF36EDB50F8
:1020800004E0D890F336E806FCE1F3508C1221D03E
:10209000450E2E6EDF502E5C1AE1020EDB500CE175
:1020A000010EF36EDB5004E0D890F336E806FCE155
:1020B000F350F31C8D160DD0010EF36EDB5004E0CF
:1020C000D890F336E806FCE1F3508D1202D00D8C67
:1020D00002D028EC0BF0030EE15C02E2E16AE5526B
:1020E000E16EE552E7CFD9FF120028EF0BF028EFA1
:1020F0000BF028EF0BF0D9CFE6FFE1CFD9FF040EAC
:10210000E126E66AD9CFE6FFDACFE6FF050EE66EF6
:1021100074EC15F0E552E552E552E552E66AD95005
:10212000010FE66E000EDA20E66E010EE66E74EC2C
:1021300015F0E552E552E552E552E66AD950020F34
:10214000E66E000EDA20E66E030EE66E74EC15F015
:10215000E552E552E552E5520D5076E1D950020FB5
:10216000E96EDACFEAFF720ED880EE542E0EED54EF
:1021700041E3D950020FE96EDACFEAFFEE50ED10DD
:102180001FE031683268336A2D0EE76E020EDBCF36
:1021900034F0030EDBCF35F0E7503426000E352245
:1021A000366A3450315C2E6E355032582F6E3650B0
:1021B0003358306E020E2EC0DBFF030E2FC0DBFF44
:1021C000010EDB50070816E3410E2E6EDF502E5C29
:1021D00002E1DF6A11D0420E2E6EDF502E5C02E16A
:1021E000080E06D0430E2E6EDF502E5C03E1100E5B
:1021F000DF6E02D00D8C28D0010EDB50DF24E96E9B
:10220000EA6AD890E936EA36690EE926010EEA2232
:10221000020EDBCFEEFF030EDBCFEDFF010EDB5036
:10222000DF24EA6A510FE96E010EEA22EF040AE1A7
:10223000010EDB50DF24EA6A510FE96E010EEA223B
:10224000020EEF6E28EC0BF0040EE15C02E2E16A94
:10225000E552E16EE552E7CFD9FF1200D9CFE6FF94
:10226000E1CFD9FF050EE126E66AD9CFE6FFDACF46
:10227000E6FF010EE66E74EC15F0E552E552E5520C
:10228000E552E66AD950020FE66E000EDA20E66EDD
:10229000010EE66E74EC15F0E552E552E552E5529A
:1022A000E66AD950030FE66E000EDA20E66E010EE4
:1022B000E66E74EC15F0E552E552E552E552E66A39
:1022C000D950010FE66E000EDA20E66E010EE66EC2
:1022D00074EC15F0E552E552E552E552E66AD95044
:1022E000040FE66E000EDA20E66E010EE66E74EC68
:1022F00015F0E552E552E552E5520D5012E1DFCFFF
:10230000C0F2020EDBCFC2F2010EDBCFC1F2030E30
:10231000DBCFC3F2040EDBCFC4F2C0C289FF28ECCE
:102320000BF0050EE15C02E2E16AE552E16EE55276
:10233000E7CFD9FF1200D9CFE6FFE1CFD9FF040ED6
:10234000E126030EDB6A0201C851EA6A000FE96E5A
:10235000030EEA22EF502C081DE00201C851EA6A80
:10236000000FE96E030EEA22EF50E66EE66A2A0ECF
:102370002E6E530E2F6E306A2EC0E6FF2FC0E6FF82
:1023800030C0E6FFF6EC2BF0316E050EE15E315009
:102390000D8A20D10201C82B0201C8512E6E2F6A6E
:1023A000000E2E1802E1010E2F1802E10201C86B87
:1023B000C0C289FF0201C11D89142E6E891C020151
:1023C000C1152E10E76E010EE7CFDBFF0201C851E9
:1023D000EA6A000FE96E030EEA22EF500D0801E1F0
:1023E000F7D00201C851EA6A000FE96E030EEA2233
:1023F000EF50E66EE66AFDEC2CF0E552E552020E77
:10240000F3CFDBFF300EF36E020EDBCFF4FFF350A1
:10241000F45C0FE3020EDB5039080BE3300E2E6E36
:10242000020EDBCFE7FF2E50E75E020EE7CFDBFFA9
:1024300019D0410EF36E020EDBCFF4FFF350F45CC3
:102440000FE3020EDB5046080BE3370E2E6E020E32
:10245000DBCFE7FF2E50E75E020EE7CFDBFF02D0B7
:102460000D8CB8D0020EDB38F00BDF6E0201C82BEA
:102470000201C8512E6E2F6A000E2E1802E1010EC5
:102480002F1802E10201C86B0D0E2E6E0201C85119
:10249000EA6A000FE96E030EEA22EF502E5C02E1B9
:1024A0000D8898D00201C851EA6A000FE96E030E48
:1024B000EA22EF50E66EE66AFDEC2CF0E552E552BA
:1024C000020EF3CFDBFF300EF36E020EDBCFF4FF14
:1024D000F350F45C0FE3020EDB5039080BE3300ECF
:1024E0002E6E020EDBCFE7FF2E50E75E020EE7CF27
:1024F000DBFF19D0410EF36E020EDBCFF4FFF35079
:10250000F45C0FE3020EDB5046080BE3370E2E6E31
:10251000020EDBCFE7FF2E50E75E020EE7CFDBFFB8
:1025200002D00D8C57D0020EDB50DF24DF6E02018B
:10253000C82B0201C8512E6E2F6A000E2E1802E120
:10254000010E2F1802E10201C86BDF508A6E010EE6
:10255000DB50896E0201C45105E0C4C2E6FF84EC81
:102560002DF0E552C0C289FF0201C35130E0030ED5
:10257000C3C2DBFF0201C0510201C2152E6E02016F
:10258000C25180142E5C0BE1030EDB5008E000000A
:102590000000000000000000030EDB06EBD7030E76
:1025A000C3C2DBFF0201C0510201C2152E6E02013F
:1025B000C25180142E5C0BE0030EDB5008E00000DB
:1025C0000000000000000000030EDB06EBD7FED683
:1025D00028EC0BF0040EE15C02E2E16AE552E16EE8
:1025E000E552E7CFD9FF1200D9CFE6FFE1CFD9FFFF
:1025F000050EE126030EDB6A040EDB6AE66AD9509B
:10260000040FE66E000EDA20E66E010EE66E6CDA5E
:10261000E552E552E552E552040EDB5004E0040EAB
:10262000DB50380802E20D8CA4D00201C851EA6ADE
:10263000000FE96E030EEA22EF502C081DE00201A4
:10264000C851EA6A000FE96E030EEA22EF50E66E07
:10265000E66A2A0E2E6E530E2F6E306A2EC0E6FFEB
:102660002FC0E6FF30C0E6FFF6EC2BF0316E050E12
:10267000E15E31500D8A7DD00201C82B0201C851A4
:102680002E6E2F6A000E2E1802E1010E2F1802E1A5
:102690000201C86BC0C289FF0201C11D89142E6EE0
:1026A000891C0201C1152E10E76E010EE7CFDBFF7A
:1026B000040EDB505CE00201C851EA6A000FE96ECB
:1026C000030EEA22EFCFDFFF0201C82B0201C8513F
:1026D0002E6E2F6A000E2E1802E1010E2F1802E155
:1026E0000201C86B040EDB06DF508A6E010EDB5060
:1026F000896E0201C45105E0C4C2E6FF84EC2DF0EE
:10270000E552C0C289FF0201C35130E0030EC3C2CB
:10271000DBFF0201C0510201C2152E6E0201C2513F
:1027200080142E5C0BE1030EDB5008E0000000007B
:10273000000000000000030EDB06EBD7030EC3C24F
:10274000DBFF0201C0510201C2152E6E0201C2510F
:1027500080142E5C0BE0030EDB5008E0000000004C
:10276000000000000000030EDB06EBD7A1D728EC29
:102770000BF0050EE15C02E2E16AE552E16EE55222
:10278000E7CFD9FF120028EF0BF028EF0BF028EF6E
:102790000BF028EF0BF028EF0BF028EF0BF0D9CF60
:1027A000E6FFE1CFD9FF060EE126E66AD950020F17
:1027B000E66E000EDA20E66E030EE66E95D9E5525F
:1027C000E552E552E552D950020FE96EDACFEAFF41
:1027D000EE50ED1012E1010EE66ED950040FE66ED8
:1027E000000EDA20E66E050EE66E7ED9E552E55261
:1027F000E552E552010EE66E0FD0E66AD950040F9D
:10280000E66E000EDA20E66E050EE66E6DD9E55234
:10281000E552E552E552E66AD950050FE66E000E24
:10282000DA20E66E010EE66E5FD9E552E552E5521A
:10283000E5520D5001E04ED1D950020FE96EDACFCA
:10284000EAFFEE50ED1003E1B190A09241D1020EEB
:10285000DBCF2EF0030EDBCF2FF0640E2E5C000ECC
:102860002F5802E2800E01D0010E186E050EDB50CB
:10287000070801E2FFD018503A6E3B6A3C6A3D6A95
:10288000020EDBCF36F0030EDBCF37F0386A396A41
:10289000D890363637363836393636C020F037C01D
:1028A00021F038C022F039C023F018C025F03BC019
:1028B00026F03CC027F03DC028F0C5EC2CF01CC031
:1028C00032F01DC033F01EC034F01FC035F02E6A48
:1028D0001B0E2F6EB70E306E316A2EC020F02FC047
:1028E00021F0226E31C023F01CC025F01DC026F05F
:1028F0001EC027F01FC028F03FEC2AF020C0DEFFEA
:1029000021C0DDFFDECF2EF0DDCF2FF0120E2E5CCA
:10291000000E2F5804E2120EDE6EDD6A0CD0DECF00
:102920002EF0DDCF2FF0120E2E5E000E2F5A2EC08D
:10293000DEFF2FC0DDFF0101996B9A6B9B6B410E8F
:102940002E6E040EDB502E5C19E1010EF36E050EA7
:10295000DB5004E0D890F336E806FCE1F350F31CBA
:102960009216010EF36E050EDB5004E0D890F3369C
:10297000E806FCE1F350010199137ED0420E2E6E61
:10298000040EDB502E5C19E1010EF36E050EDB50D8
:1029900004E0D890F336E806FCE1F350F31C9316FC
:1029A000010EF36E050EDB5004E0D890F336E80616
:1029B000FCE1F35001019A135FD0430E2E6E040E1A
:1029C000DB502E5C19E1010EF36E050EDB5004E0C6
:1029D000D890F336E806FCE1F350F31C9416010E90
:1029E000F36E050EDB5004E0D890F336E806FCE108
:1029F000F35001019B1340D0440E2E6E040EDB50A9
:102A00002E5C19E1010EF36E050EDB5004E0D89048
:102A1000F336E806FCE1F350F31C9516010EF36E55
:102A2000050EDB5004E0D890F336E806FCE1F350E5
:102A300001019C1321D0450E2E6E040EDB502E5C3E
:102A400019E1010EF36E050EDB5004E0D890F33669
:102A5000E806FCE1F350F31C9616010EF36E050E2A
:102A6000DB5004E0D890F336E806FCE1F3500101B6
:102A70009D1302D00D8C2ED031683268336ADECFC0
:102A800034F0DDCF35F0366A3450315C2E6E35507F
:102A900032582F6E36503358306E2EC0DEFF2FC0A6
:102AA000DDFFDECF2EF0DDCF2FF02FC02EF02F6A0E
:102AB0002E50166EDECF2EF0DDCF2FF02E50176E7B
:102AC000196AB192B198B19AA282A192A082B18002
:102AD00028EC0BF0060EE15C02E2E16AE552E16EE1
:102AE000E552E7CFD9FF1200D9CFE6FFE1CFD9FFFA
:102AF000040EE126030EDB6A0D0E2E6E0201C85194
:102B0000EA6A000FE96E030EEA22EF502E5C05E13F
:102B1000FB0EDB5044E10D8842D0C851EA6A000F39
:102B2000E96E030EEA22EF502C081FE0FB0EDB508B
:102B30001AE1C851EA6A000FE96E030EEA22EF506B
:102B4000E66EE66A2A0E2E6E530E2F6E306A2EC087
:102B5000E6FFE66E30C0E6FFF6EC2BF0316E050EB8
:102B6000E15E31500D8A020E90D1C82BC8512E6EF5
:102B70002F6A000E2E1804E1010E2F1801E1C86B18
:102B80000D0E2E6EC851EA6A000FE96E030EEA229E
:102B9000EF502E5C06E1FB0EDB5001E10D88030EC9
:102BA00074D12D0E2E6EC851EA6A000FE96E030E25
:102BB000EA22EF502E5C27E1040E2F6EFE0EDB5052
:102BC0002F5C21E0050E306EFE0EDB50305C1BE00A
:102BD000FE0EDB0401E12FD1030E2E6EFE0EDB5044
:102BE0002E5C01E128D1010EF36E030EF3CFDBFF63
:102BF000C82BC8512E6E2F6A000E2E1804E1010E4C
:102C00002F1801E1C86B040E2E6EFE0EDB502E5CF9
:102C100011E0050E2F6EFE0EDB502F5C0BE0050E53
:102C2000E66ED9CFE6FFDACFE6FF3BD9E552E552B3
:102C3000E5523DD0C851EA6A000FE96E030EEA2260
:102C4000EFCF2EF02F6A306A2EC0DFFF010E2FC0AB
:102C5000DBFF020E30C0DBFF050E2E6EFE0EDB50DA
:102C60002E5C19E1000EDFCFE6FF010EDBCFE6FFA1
:102C7000FDEC2CF0E552E552F3CF2EF0F4CF2FF01F
:102C8000306A2FBE30682EC0DFFF010E2FC0DBFF81
:102C9000020E30C0DBFF0201C82BC8512E6E2F6A16
:102CA000000E2E1804E1010E2F1801E1C86B030E6F
:102CB000DB501DE0DFCF2EF0010EDBCF2FF0020E38
:102CC000DBCF30F02668276828682EC021F02FC09F
:102CD00022F030C023F073EC2AF01EC02EF01EC08C
:102CE000DFFF010E1FC0DBFF020E20C0DBFFFE0E68
:102CF000DB5026E1DFCF2EF0010EDBCF2FF0020EEE
:102D0000DBCF30F03034000E301807E6D8807F0E6D
:102D10002E54000E2F54000E305401E28CD0D9CF27
:102D2000E9FFDACFEAFF020ED880EB50FF0A06E691
:102D3000800EEE5CFF0EEE58FF0EEF5801E27BD0E6
:102D4000FE0EDB0424E1DFCF31F0010EDBCF32F0E9
:102D5000020EDBCF33F03334000E331807E6D88091
:102D6000FF0E3154000E3254000E335464E3D9CFB9
:102D7000E9FFDACFEAFF020ED890EB50000A06E630
:102D8000000EEE5C000EEE58000EEF5854E3020EFB
:102D9000346EFE0EDB50345C24E1DFCF35F0010EE3
:102DA000DBCF36F0020EDBCF37F03734000E3718AA
:102DB00007E6D880FF0E35547F0E3654000E375488
:102DC0003AE3D9CFE9FFDACFEAFF020ED880EB5021
:102DD000FF0A06E6000EEE5C800EEE58FF0EEF587E
:102DE0002AE3030E386EFE0EDB50385C27E1DFCF9E
:102DF00039F0010EDBCF3AF0020EDBCF3BF03B3473
:102E0000000E3B1807E6D880FF0E3954FF0E3A54E7
:102E1000000E3B5410E3D9CFE9FFDACFEAFF020EF0
:102E2000D890EB50000A06E6000EEE5C000EEE585D
:102E3000000EEF5803E20D8C010E27D0FE0EDB5082
:102E4000030A16E0010A14E0030A08E0050A06E096
:102E5000010A04E0050A02E0040E17D0FC0EDBCFE5
:102E6000E9FFFD0EDBCFEAFF000EDFCFEFFF0CD056
:102E7000FC0EDBCFE9FFFD0EDBCFEAFF000EDFCF5C
:102E8000EEFF010EDBCFEDFF000E2E6E040EE15CB7
:102E900002E2E16AE552E16E2E50E552E7CFD9FF3A
:102EA0001200D9CFE6FFE1CFD9FF020EE126FD0ED9
:102EB000DBCFE9FFFE0EDBCFEAFFEE6AEE6AEE6AD9
:102EC000010EDB6AFC0EDB50F36E010EDBCFF4FF6C
:102ED000F350F45C53E20201C851EA6A000FE96E54
:102EE000030EEA22EFCFDFFF300EDF5C42E3DF505C
:102EF00039083FE3FD0EDBCFE9FFFE0EDBCFEAFF33
:102F0000EECF31F0EECF32F0EFCF33F00A0E266E77
:102F1000276A286A31C021F032C022F033C023F082
:102F200073EC2AF0300EDF5C346E356A366A1E5060
:102F300034242E6E1F5035202F6E20503620306ED8
:102F4000FD0EDBCFE9FFFE0EDBCFEAFF2EC0EEFF6A
:102F50002FC0EEFF30C0EEFF0201C82BC8512E6E0D
:102F60002F6A000E2E1807E1010E2F1804E1C86B1E
:102F700002D0000E04D0010EDB2AA4D7010E2E6E63
:102F8000020EE15C02E2E16AE552E16E2E50E5528A
:102F9000E7CFD9FF12000650E66EE66A1E0E2E6ECF
:102FA000530E2F6E306A2EC0E6FFE66E30C0E6FF8D
:102FB000F6EC2BF0316E050EE15E3150120000018F
:102FC000605108E0010E2E6E6D50020B01E0010E03
:102FD0002E5C1BE10101E807000EE95BEA510BE101
:102FE000E851E91111E18B80D00EE86F070EE96F0F
:102FF000010EEA6F1200E851E9114DE18B90D00EFD
:10300000E86F070EE96FEA6B1200600509E0020E37
:10301000605D06E0040E605D03E0100E605D02E19D
:103020008B801200200E605D36E10101E807000E82
:10303000E95BEA510AE1E851E9112DE18B80100EBC
:10304000E86F270EE96F010E18D0EA050AE1E85192
:10305000E91121E18B90100EE86F270EE96F020E47
:103060000CD0020EEA5D0BE1E851E91114E18B800E
:10307000A00EE86F860EE96F030EEA6F1200030ED2
:10308000EA5D09E3E851E91106E18B90100EE86F63
:0E309000270EE96FEA6B120082A4010C000CFF
:02309E00D9CF88
:1030A000E6FFE1CFD9FFE652A09A6A6A686A706AC1
:1030B000030EE66EE66AE66A710EE66E0F0EE66EC7
:1030C000A9EC2BF02E6E050EE15E2E50160E6F6EE3
:1030D0009F0E6B6E7B0E696EDF6ADF502E6E2F6A5D
:1030E000100E2E5C000E2F5810E2DF50040DF3CFAF
:1030F000E9FFF4CFEAFF000EE926040EEA22EE6AA9
:10310000EE6AEE6AEE6ADF2AE8D76D8C6E6A6D9819
:103110006D9C68A607D0689600017B6B806B816B05
:10312000826BF7D70001010E966F976F986B996BC2
:10313000886BDF6A040EDF5C26E2EA6ADF34FE0B8E
:10314000EA36E96E6F0EE926000EEA22EE6AED6AB3
:10315000EA6ADF34FE0BEA36E96E670EE926000EF6
:10316000EA22EE6AED6ADF50EA6A8C0FE96E000E21
:10317000EA22EF6ADF50EA6A900FE96E000EEA2257
:10318000EF6ADF2AD7D70001080E6F6F040E706F49
:10319000160E706E0401400E026F040E036F400E97
:1031A000016F840E006F0001616B606BE552E552A8
:1031B000E7CFD9FF1200D9CFE6FFE1CFD9FFE65222
:1031C0000001600507E16DBA05D0686A6980698809
:1031D000020E606F6850040B05E06950040B02E0BA
:1031E0006894BFD86DB250D06850010B09E06950A7
:1031F000010B06E054DFA08A0001040E606F6890A6
:103200006850100B05E06950100B02E095D86898E3
:1032100068AC12D069AC0FD0010EE66EE66A000E03
:10322000E66EE66A730EE66EE66A0FEC2BF02E6E23
:10323000060EE15E2E50689C6850200B04E0695039
:10324000200B01E060D86850020B13E06950020BBC
:1032500010E0010EE66EE66A000EE66EE66AE668CB
:103260007F0EE66E0FEC2BF02E6E060EE15E2E50FA
:103270006A6A040E0001E76E6019E8AE02D0E73416
:1032800002D0E750605D02E2A19A38D069A635D03D
:10329000DF6A040EDF5C31E268A62FD06CCF89F0C4
:1032A00000018951780BE842E842E8428A6F68964B
:1032B00089B506D08A51EA6A900FE96E000E05D0F2
:1032C0008A51EA6A8C0FE96E000EEA22EF708A5189
:1032D00002E15ED810D0000EE66EE66A890EE66E58
:1032E000000EE66E720EE66EE66A0FEC2BF02E6EA6
:1032F000060EE15E2E50DF2ACCD7A19AE552E552A8
:10330000E7CFD9FF120070A015D063C0E9FF64C0F9
:10331000EAFFEF5080080DE16FC0E9FF70C0EAFFDF
:10332000EF50840806E163C0E9FF64C0EAFF8C0E39
:10333000EF6E7090689A1200698468986D8200013F
:10334000010E886F000EE66EE66AE66EE66A750E9E
:10335000E66EE66A0FEC2BF02E6E060EE15E2E5046
:1033600012000001886B000EE66EE66AE66EE66A01
:10337000740EE66EE66A0FEC2BF02E6E060EE15E22
:103380002E506D92699468A402D06894FCD7120004
:10339000D9CFE6FFE1CFD9FFE652FD0E0001891536
:1033A00053E17E0E8915E8407F0B040DF3CF63F0E7
:1033B000F4CF64F0000E6327040E642363C065F04D
:1033C00064C066F0657563C0E9FF64C0EAFFEF5052
:1033D0003C0BE842E8420D0835E1DF6A080EDF5C8D
:1033E00023E263C0E9FF64C0EAFF020EE926000E93
:1033F000EA22EE50EFCFEAFFE96EEF50E66EDF50C3
:10340000EA6A400FE96E040EEA22E552E750EF6ED9
:1034100063C0E9FF64C0EAFF020EE926000EEA225B
:10342000EE2AEF22DF2ADAD763C0E9FF64C0EAFFA1
:10343000020EE926000EEA22400EEE6E040EED6E3C
:103440000DD807D03AD805D0FD0E8915040801E142
:1034500059D8E552E552E7CFD9FF12000001776B4A
:10346000956B986B996B8B6B786B6FC0E9FF70C035
:10347000EAFFEF9E6F756FC0E9FF70C0EAFFEF9E35
:103480006F7565C0E9FF66C0EAFFEF9E7B6B7C6BE2
:103490007D6B806B816B826B8CD8000EE66EE66A6A
:1034A000E66EE66A030EE66EE66A0FEC2BF02E6E11
:1034B000060EE15E2E50A8EF1DF0020E0001785DB1
:1034C00002E168EF1EF0786B8B511AE165C0E9FFED
:1034D00066C0EAFFEE52400EEF6E65C0E9FF66C0BF
:1034E000EAFF020EE926000EEA22400EEE6E040EFE
:1034F000ED6E65C0E9FF66C0EAFF8C0EEF6E12004C
:103500008B6B1200D9CFE6FFE1CFD9FFE6526FC037
:10351000E9FF70C0EAFFEF50400B01E0010EDF6EE3
:1035200000016F75080E605D08E142C46EFF6E50C9
:1035300002E0100E01D0040E606F780526E16FC026
:10354000E9FF70C0EAFF020EE926000EEA22480EEB
:10355000EE6E040EED6E5DDB020E0001775D06E19E
:103560006FC0E9FF70C0EAFF840E0DD0DF5006E1A6
:103570006FC0E9FF70C0EAFFC80E05D06FC0E9FF59
:1035800070C0EAFF880EEF6E0FD080AF0CD0835171
:10359000841107E005D084C0FAFF00018351F96E61
:1035A000FADF0001809F786BE552E552E7CFD9FF43
:1035B000120004014051600BE842E842E842E84250
:1035C000E842000901E0120041510C0A50E00B0AE8
:1035D0003FE00C0A31E0010A22E00B0A1EE0020A79
:1035E0001CE0030A18E0080A10E0010A0CE00F0AC8
:1035F00008E0030A01E0120000017B8F080E606FF3
:103600001200F1EF1CF007EF1FF00001610E796F5F
:10361000000E7A6F0CD04EEF1DF038EF1BF04451C6
:103620000001796F7A6B620E7927000E7A237B8115
:10363000010E7C6F7B8F120000017B8F04014451CF
:10364000EA6A620FE96E000EEA2242C4EFFF12003E
:10365000000EE66EE66AE66EE66A020EE66EE66A60
:103660000FEC2BF02E6E060EE15E2E5012001200B3
:10367000D9CFE6FFE1CFD9FF030EE12604014205D1
:1036800010E140511F0B00090CE100017B8F030E7C
:103690000401415D04E10001010E876F02D00001C9
:1036A000876B0401425101E003D140511F0B020816
:1036B00001E0FED044510F0B000901E1F9D0445163
:1036C0000F0B030801E2F4D0200E0001605D01E061
:1036D000EFD07B8F040144BF16D044510F0BE96E2D
:1036E000EA6AD890E936EA36670EE926000EEA2241
:1036F000EECFDEFFEDCFDDFF44510F0BEA6A900FF6
:10370000E96E000E15D044510F0BE96EEA6AD890AD
:10371000E936EA366F0EE926000EEA22EECFDEFF2A
:10372000EDCFDDFF44510F0BEA6A8C0FE96E000EFE
:10373000EA22020EEFCFDBFFD950020FE96EDACF9B
:10374000EAFFEF50010B03E1000EDF9401D0DF84AC
:1037500044BF0BD044510F0BE96EEA6AD890E936AA
:10376000EA36670EE926000E0AD044510F0BE96EC7
:10377000EA6AD890E936EA366F0EE926000EEA22A8
:10378000DECFEEFFDDCFEDFF030E415D20E1DECFAA
:10379000E9FFDDCFEAFFEF50800B11E044BF07D017
:1037A00044510F0BEA6A900FE96E000E06D04451A7
:1037B0000F0BEA6A8C0FE96E000EEA22EF82840E8C
:1037C000DECFE9FFDDCFEAFFE850EF1271D0DF7402
:1037D000DECFE9FFDDCFEAFFEF50800B1BE0DECF4D
:1037E000E9FFDDCFEAFFEF9EDECFE9FFDDCFEAFFA5
:1037F000EF8C020EE66EE66ADECFE6FFDDCFE6FF77
:10380000050EE66EE66A0FEC2BF02E6E060EE15EFC
:103810002E5005D0DECFE9FFDDCFEAFFEF8CDF745D
:10382000D950020FE96EDACFEAFFEF50020B0EE13A
:10383000DECFE9FFDDCFEAFFEF50800B32E0DECFD5
:10384000E9FFDDCFEAFFEF50040B2BE1040144BF99
:1038500007D044510F0BEA6A900FE96E000E06D0B4
:1038600044510F0BEA6A8C0FE96E000EEA22EF92C8
:103870003B0E2E6EDECFE9FFDDCFEAFFE850EF16FC
:10388000020EE66EE66ADECFE6FFDDCFE6FF050E4E
:10389000E66EE66A0FEC2BF02E6E060EE15E2E5001
:1038A00007D03B0EDECFE9FFDDCFEAFFE850EF1691
:1038B000030EE15C02E2E16AE552E16EE552E7CF18
:1038C000D9FF1200000196514DE1010E966F9751FC
:1038D00049E1010E976F020E785D0DE16FC0E9FFBF
:1038E00070C0EAFFEE52EF6A6FC0E9FF70C0EAFFF6
:1038F000C80EEF6E1200780535E18B6B63C0E9FFEF
:1039000064C0EAFFEE52400EEF6E63C0E9FF64C090
:10391000EAFF020EE926000EEA22400EEE6E040EC9
:10392000ED6E63C0E9FF64C0EAFF840EEF6E010E26
:103930008B6F65C0E9FF66C0EAFFEE52400EEF6E86
:1039400065C0E9FF66C0EAFF020EE926000EEA2222
:10395000400EEE6E040EED6E65C0E9FF66C0EAFF34
:10396000800EEF6E12000001986B996B020E785D6D
:1039700018E165C0E9FF66C0EAFFEE52400EEF6E47
:1039800065C0E9FF66C0EAFF020EE926000EEA22E2
:10399000480EEE6E040EED6E65C0E9FF66C0EAFFEC
:1039A0001DD07C510401465D00017D510401475941
:1039B00004E246C47CF047C47DF02BD96FC0E9FF18
:1039C00070C0EAFF020EE926000EEA22480EEE6EF3
:1039D000040EED6E6FC0E9FF70C0EAFFC80EEF6E17
:1039E0001200800E0401405D58E10001C00E7B6FA3
:1039F00004014351030A2FE0010A09E0030A4BE1E5
:103A00000001080E796F590E7A6F120E3ED04251A6
:103A1000F66EF76AD890F636F736810EF626590E0E
:103A2000F7220900F5CF79F00A00F5CF7AF0020EFF
:103A30000001F76A7925F66E7A51F7220800F5CF72
:103A40007CF0030EF76A7925F66E7A51F7220800AA
:103A5000F5CF7DF01200030E425D1AE24251F66E80
:103A6000F76AD890F636F736830EF626590EF72207
:103A70000900F5CF79F00A00F5CF7AF079C0F6FFAA
:103A80007AC0F7FF0800F55000017C6F7D6B1200D3
:103A900000017B6B120000017B6B1200D9CFE6FFA7
:103AA000E1CFD9FF020EE1260401486B496B40517A
:103AB0001F0B020A11E0030A0CE0010A35E10001C4
:103AC0007B8F04014881000187052EE104014883B2
:103AD0002BD000017B8F28D000017B8F040144BFD5
:103AE0000BD044510F0BE96EEA6AD890E936EA36FA
:103AF000670EE926000E0AD044510F0BE96EEA6A00
:103B0000D890E936EA366F0EE926000EEA22EECFAB
:103B1000DEFFEDCFDDFFDECFE9FFDDCFEAFFEF50C7
:103B2000040B02E0010E486F00017BAF07D0480E86
:103B3000796F040E7A6F7B81020E7C6F020EE15C5E
:103B400002E2E16AE552E16EE552E7CFD9FF1200E9
:103B50006D9800017BBF2BD080AF09D0020E786F2B
:103B6000995101E100DF0001976B966B120065C06F
:103B7000E9FF66C0EAFFEE52400EEF6E65C0E9FF56
:103B800066C0EAFF020EE926000EEA22400EEE6E43
:103B9000040EED6E65C0E9FF66C0EAFF8C0EEF6EA5
:103BA0006FC0E9FF70C0EAFF840EEF6E12000401DF
:103BB00040AF0DD00001010E786F985101E1D3DEC6
:103BC0000001976B966B955123E162EF1CF00001A9
:103BD000020E786F65C0E9FF66C0EAFFEE52400E44
:103BE000EF6E65C0E9FF66C0EAFF020EE926000E2F
:103BF000EA22400EEE6E040EED6E65C0E9FF66C06F
:103C0000EAFF840EEF6E976B966B955101E15ADED9
:103C10001200D9CFE6FFE1CFD9FFE652400EDF6EAA
:103C200000017C5D000E7D590AE27CC0DFFF775108
:103C300002E1010E03D0770502E1020E776FDF503B
:103C40002F6AE8507C5D7C6F2F507D597D6F6FC06F
:103C5000E9FF70C0EAFFEE52DFCFEFFF480E856F3D
:103C6000040E866F7BB118D0DF502DE079C0F6FFCF
:103C70007AC0F7FF792B000E7A230800F550E66E24
:103C800085C0E9FF86C0EAFF852B000E8623E5523A
:103C9000E750EF6EDF06E8D7DF5015E079C0E9FFA7
:103CA0007AC0EAFF792B000E7A23EF50E66E85C0CA
:103CB000E9FF86C0EAFF852B000E8623E552E75018
:103CC000EF6EDF06E9D7E552E552E7CFD9FF1200E4
:103CD000D9CFE6FFE1CFD9FF020EE12663C0E9FFAD
:103CE00064C0EAFFEE52EFCFDFFFDFCF2EF02E50A1
:103CF0000001815D000E825902E281C0DFFFDF50CA
:103D00002E6E2F6AE850815D816F2F508259826F2D
:103D1000010EDB6ADF50F36E010EDBCFF4FFF350D0
:103D2000F45C16E2010EDB50EA6A480FE96E040EFD
:103D3000EA22EF50E66E7EC0E9FF7FC0EAFF7E2BED
:103D4000000E7F23E552E750EF6E010EDB2AE2D72B
:103D5000000ED8808155000E825527E265C0E9FF2C
:103D600066C0EAFFEE52400EEF6E65C0E9FF66C026
:103D7000EAFF020EE926000EEA22480EEE6E040E5D
:103D8000ED6E63C0E9FF64C0EAFFEF50400B06E14F
:103D900065C0E9FF66C0EAFFC80E05D065C0E9FF4F
:103DA00066C0EAFF880EEF6E28D065C0E9FF66C0E6
:103DB000EAFFEE52400EEF6E65C0E9FF66C0EAFF13
:103DC000020EE926000EEA22400EEE6E040EED6EA3
:103DD00065C0E9FF66C0EAFF840EEF6E835184116F
:103DE00007E005D084C0FAFF00018351F96EFADFC5
:103DF0000001809F955101E165DD020EE15C02E268
:103E0000E16AE552E16EE552E7CFD9FF1200D9CF62
:103E1000E6FFE1CFD9FFE65200017B8F030EE66E8D
:103E2000E66AE66A710EE66E0F0EE66EA9EC2BF0FE
:103E30002E6E050EE15E2E50DF6ADF502E6E2F6A69
:103E4000100E2E5C000E2F5810E2DF50040DF3CF41
:103E5000E9FFF4CFEAFF000EE926040EEA22EE6A3B
:103E6000EE6AEE6AEE6ADF2AE8D76D8C010EE66E26
:103E7000E66AE66A620EE66E000EE66EA9EC2BF0CC
:103E80002E6E050EE15E2E506D9C0001080E6F6FC8
:103E9000040E706F000E636F040E646F63C065F0F4
:103EA000666F42C461F0615102E1100E12D0010E42
:103EB000E66EE66A610EE66E000EE66E010EE66ED6
:103EC000E66A0FEC2BF02E6E060EE15E2E5000011E
:103ED000200E606FE552E552E7CFD9FF1200D9CF2F
:103EE000E6FFE1CFD9FF020EE126000EDE6E040EE2
:103EF000DD6EFD0EDB50E824306EFE0EDB50040D4F
:103F0000F3503024040DF4CF2FF0D9CFE9FFDACFEE
:103F1000EAFFF350EE262F50ED22DECFE9FFDDCF92
:103F2000EAFFEF9EFD0EDB500AE1FE0EEA6ADB348B
:103F3000FE0BEA36E96E670EE926000E09D0FE0E8A
:103F4000EA6ADB34FE0BEA36E96E6F0EE926000EF4
:103F5000EA22DECFEEFFDDCFEDFFDECFE9FFDDCFE2
:103F6000EAFFEF9CDECFE9FFDDCFEAFF040EE92692
:103F7000000EEA22EF8C020EE15C02E2E16AE552F9
:103F8000E16EE552E7CFD9FF1200D9CFE6FFE1CFCE
:103F9000D9FF020EE126FD0EDBA407D0E66AFE0E75
:103FA000DBCFE6FF9CDFE552E552FD0EDBA208D039
:103FB000010EE66EFE0EDBCFE6FF91DFE552E55225
:103FC000FE0EDB502F6A700F2E6E0F0E2F222EC0AA
:103FD000DEFF2FC0DDFFDECFE9FFDDCFEAFFFD0E04
:103FE000DBCFEFFF020EE15C02E2E16AE552E16E37
:103FF000E552E7CFD9FF1200D9CFE6FFE1CFD9FFD5
:10400000020EE126FE0EDB5020E165C0E9FF66C02E
:10401000EAFFEE52400EEF6E65C0E9FF66C0EAFFB0
:10402000020EE926000EEA22400EEE6E040EED6E40
:1040300065C0E9FF66C0EAFF8C0EEF6E6FC0E9FF56
:1040400070C0EAFF840EEF6E3BD0FD0EDB50E8241B
:10405000306EFE0EDB50040DF3503024040DF3CF10
:104060002EF0F4CF2FF0000E2E26040E2F222EC09D
:10407000DEFF2FC0DDFF840EDECFE9FFDDCFEAFFDC
:10408000E850EF12FD0EDB50E824306EFE0EDB50E0
:10409000040DF3503024010F040DF3CF2EF0F4CFB4
:1040A0002FF0000E2E26040E2F222EC0DEFF2FC072
:1040B000DDFF840EDECFE9FFDDCFEAFFE850EF122F
:1040C000020EE15C02E2E16AE552E16EE552E7CF01
:1040D000D9FF1200D9CFE6FFE1CFD9FF020EE126CA
:1040E000FD0EDB500AE0FE0EEA6ADB34FE0BEA3618
:1040F000E96E6F0EE926000E09D0FE0EEA6ADB3487
:10410000FE0BEA36E96E670EE926000EEA22EECFD4
:10411000DEFFEDCFDDFFD9CFE9FFDACFEAFFEE50CA
:10412000ED1003E1F36AF46A44D0DECFE9FFDDCF9E
:10413000EAFF020EE926000EEA22FB0EDBCFEEFFBD
:10414000FC0EDBCFEDFFDECFE9FFDDCFEAFFEE5265
:10415000FA0EDBCFEFFF400EDECFE9FFDDCFEAFF47
:10416000E850EF16880EDECFE9FFDDCFEAFFE8501A
:10417000EF12FD0EDB500AE0FE0EEA6ADB34FE0BA6
:10418000EA36E96E6F0EE926000E09D0FE0EEA6AE5
:10419000DB34FE0BEA36E96E670EE926000EEA22F2
:1041A000EF74DECF2EF0DDCF2FF02EC0F3FF2FC047
:1041B000F4FF020EE15C02E2E16AE552E16EE552D3
:1041C000E7CFD9FF1200D9CFE6FFE1CFD9FF6DA825
:1041D0004ED0FE0EEA6ADB34FE0BEA36E96E6F0E55
:1041E000E926000EEA22EE50EFCFEAFFE96E400E1C
:1041F000EE16EE6AEE6AEE6AFE0EEA6ADB34FE0B3B
:10420000EA36E96E6F0EE926000EEA22EE50EFCF95
:10421000EAFFE96EEE7CFE0EEA6ADB34FE0BEA365C
:10422000E96E6F0EE926000EEA22EF74400E2E6E44
:10423000FE0EEA6ADB34FE0BEA36E96E6F0EE92603
:10424000000EEA22EE50EFCFEAFFE96E2E50EF1695
:10425000FE0EEA6ADB34FE0BEA36E96E6F0EE926E3
:10426000000EEA22EE50EFCFEAFFE96EEF7CE55256
:10427000E7CFD9FF12006D6A696A0001606B120016
:104280000001605113E16D6A696A160E6F6E9F0E30
:104290006B6E7B0E696ED08EA29AA08AF28E6DB67E
:0E42A00002D06D86FCD70001010E606F120087
:0242AE0093EC8F
:1042B00026F0FB0EDBCFF3FFDB06F35000090AE02C
:1042C000E1EC26F0FA0E4CEC27F0F3E12F1CF1E1C3
:1042D000010E01D0000EC2EF26F093EC26F03B0E4B
:1042E000E12402E3E168E652E16E010EDB6A020EB0
:1042F000DB6AF90EDBCFF6FFFA0EDBCFF7FFFB0E22
:10430000DBCFF8FF0800F550DF6EDF5002E1E6EF8B
:1043100025F0250EDF5C02E0D9EF25F0030EDB6A05
:10432000040EDB6A050EDB6A060EDB6A070EDB6A2B
:10433000FBEC25F02D0EDF5C0CE02B0EDF5C09E0C2
:10434000200EDF5C06E0230EDF5C03E0300EDF5C56
:104350001AE1DF50300A14E0130A0FE0030A0AE002
:104360000B0A05E0060AE4E1030EDB80E1D7030E49
:10437000DB82DED7030EDB84DBD7030EDB86D8D7E8
:10438000030EDB88D5D72A0EDF5C1BE1F7EC25F0A6
:1043900045EC26F010E0030EDB8022682368130E44
:1043A000DBCF27F0140EDBCF28F0BCEC2AF0040E94
:1043B00020C0DBFF03D0130E2EEC26F0FBEC25F023
:1043C0000BD0090EDB6A9CEC26F003E010EC27F022
:1043D000FAD7090E2EEC26F0030EDBB0DB982E0E7A
:1043E000DF5C1BE1FBEC25F02A0EDF5C0BE1F7EC58
:1043F00025F045EC26F003E1130E80EC26F0FBECF3
:1044000025F00BD0090EDB6A9CEC26F003E010ECE3
:1044100027F0FAD7090E80EC26F0680EDF5C07E182
:10442000FBEC25F0680EDF5C1DE1030E18D0740E66
:10443000DF5C17E07A0EDF5C14E0480EDF5C06E01C
:10444000540EDF5C03E05A0EDF5C02E1020E07D07F
:104450006C0EDF5C03E06A0EDF5C04E1010ED3EC5E
:1044600026F0C9DBDF506E0A01E17FD31E0A01E1AD
:1044700092D1200A01E18FD13F0A01E149D11A0A04
:1044800001E146D10D0A01E143D1200A01E140D109
:104490003A0A01E13DD1200A01E13AD1260A01E1BF
:1044A00035D10D0A01E132D11A0A01E1D9D0200A31
:1044B0004AE0300A1FE0460A0EE0250A01E083D3F5
:1044C000D950F90FE96EFF0EDA20EA6E010EEE5EAA
:1044D000000EEE5AEE5AE1EC26F0250EE66E95DB64
:1044E00003E12F1C01E169D3DDEC26F001E26BD37F
:1044F000DB2A69D3080EDB6A040EDB50010806E2F2
:10450000040EDB04A5EC26F0DB508BDB080EDB5041
:1045100009E0030EDB50010B05E172DB01E04DD336
:10452000080EDB6A64DBEFCFDFFF55EC27F003E119
:104530002F1C01E142D3DDEC26F001E3DB2A60DB36
:1045400001E141D33AD3070EDB5002080FE121EC21
:1045500027F0030EE8EC26F00E0EEECFDBFF0F0E79
:10456000EECFDBFF100EEECFDBFF20D0F70EDBCF60
:1045700031F0F80EDBCF32F0020E315E000E325A0F
:10458000F70E31C0DBFFF80E32C0DBFF31C0E9FFB0
:1045900032C0EAFFD8EC26F0306A0E0E2EC0DBFFE8
:1045A0000F0E2FC0DBFF100E30C0DBFF0E0EDBCF77
:1045B000E6FF0F0EDBCFE6FF100EDBCFE6FFD1EC00
:1045C0002BF0E552E552E552130E21C0DBFF140E2D
:1045D00022C0DBFF060EDB5005E0130E1CEC27F0BB
:1045E00001E26ADB40EC27F002E2130E37DB03EC5A
:1045F00027F006E0040E1CEC27F002E2050E2EDB8D
:10460000030EDBB005D0FCDA01E0D7D2080EDB6A7E
:10461000090EDB6A0E0EDBCFF6FF0F0EDBCFF7FFC6
:10462000100EDBCFF8FF0800F550DF6EDF5014E00E
:1046300046EC27F011E255EC27F003E12F1C01E1D5
:10464000BCD2BBDB01E3DB2A090EDB2AD9500E0FFB
:10465000E96E000ECBDBE7D7D3DA01E1B4D2ADD2FD
:10466000C6DA110EEECFDBFF120EEDCFDBFF110E1F
:10467000DBCFE6FF120EDBCFE6FFC3EC2BF0E552FB
:10468000E552130EF3CFDBFF140EF4CFDBFF060E63
:10469000DB5004E0130ED0DB01E20EDB40EC27F030
:1046A00002E2130EDBDAAFDB05E0040EC5DB02E24B
:1046B000050ED4DA030EDBB005D0A2DA01E07DD21C
:1046C000080EDB6A090EDB6A110EDBCFE9FF120E62
:1046D000DBCFEAFFEFCFDFFFDF5014E0D7DB12E2E2
:1046E000E4DB03E12F1C01E168D267DB01E3DB2A95
:1046F000090EDB2A110EDB2ADBCFE9FF120EE8E3FD
:10470000DB2AE6D77DDA01E15ED257D2030EDB8EDB
:10471000070EDB0410E195DB040E5ADB0A0EEECF28
:10472000DBFF0B0EEECFDBFF0C0EEECFDBFF0D0E33
:10473000EECFDBFF6CD0070EDB5003082CE1030E3D
:10474000DBAE0DD0B2DA020E76DAEFCF2EF02F6AA2
:10475000306A316A2EAE39D02F68306835D0F70E06
:10476000DBCF2FF0F80EDBCF30F0020E2F5E000E05
:10477000305AF70E2FC0DBFFF80E30C0DBFF2FC022
:10478000E9FF30C0EAFFEFCF2EF00A0E2EC0DBFFAC
:104790000B0EDB6A38D0070EDB50020809E1030E6E
:1047A000DBAE04D059DB30AE10D00ED055DB0DD0CF
:1047B000030EDBAE12D079DA020E3DDAF9DA306A96
:1047C000316A2FAE02D030683168E2DA0C0E30C0A8
:1047D000DBFF0D0E31C0DBFF1AD0F70EDBCF30F060
:1047E000F80EDBCF31F0020E305E000E315AF70EBC
:1047F00030C0DBFFF80E31C0DBFF30C0E9FF31C055
:10480000EAFFD6DAC5DA0C0EDB6A0D0EDB6A060E9D
:10481000DB5005E1010EF36E050EF3CFDBFF150E45
:10482000DB6A160EDB6AD950370F2E6E000EDA20C7
:104830002F6E390E2EC0DBFF3A0E2FC0DBFF380E75
:10484000DB6A080EDB6A0A0EAEDADF50780A12E085
:10485000200A10E0280A0CE0200A0AE03F0A06E0DD
:104860000D0A02E0200A08E1020E05D0080E03D06E
:10487000080EDF26100E97DA030EDBBE02D0DB92A5
:10488000DB94DB50800B24E08ADAD890030EEB50E7
:10489000000A08E6000EEE5C000EEE58000EEE5820
:1048A000000EEE5815E213DA256826682768286896
:1048B000C5EC2CF00A0E1CC0DBFF0B0E1DC0DBFF8D
:1048C0000C0E1EC0DBFF0D0E1FC0DBFF2D0E08D02F
:1048D000030EDBA202D02B0E03D0DBA408D0200EE7
:1048E000F36E170EF3CFDBFF150EDB2A02D0170E87
:1048F000DB6A050EDB5003E1B7D901E189D01E0E5A
:104900002E6E5B0E2F6E000E306E070EDBCF31F079
:10491000326A336A346A31C025F032C026F033C0BF
:1049200027F034C028F0D3D923EC2DF02E501C24CE
:10493000F36E2F501D20F46E30501E20F86EF4CF11
:10494000F7FFF3CFF6FF0800090EF5CFDBFF580E97
:10495000DF5C0FE1610EF36E090E7BD90AE3200ED6
:104960002E6E090EDBCFE7FF2E50E75E090EE7CF74
:10497000DBFF070EDBCF2EF02F6A306A316A0FDAC9
:104980002EC025F02FC026F030C027F031C028F00F
:10499000EECF20F0EECF21F0EECF22F0EFCF23F0DC
:1049A00023EC2DF023C0EDFF22C0EDFF21C0EDFF71
:1049B00020C0EFFF390EDBCFE9FFDB063A0EDBCF7D
:1049C000EAFF01E2DB06090EDBCFEFFF150EDB2A63
:1049D0004BD995E1030EDBA61DD06F0EDF5C06E11F
:1049E000C1D918E3150EDB285BDA14D0780EDF5C32
:1049F00009E0580EDF5C06E0620EDF5C03E0420E69
:104A0000DF5C08E1020EF36E160EF3CFDBFF02D07F
:104A1000150EDB6A030EDB50100B0EE0040EDBCF2D
:104A20002EF0050EDB50D8802E5406E2060EDB5029
:104A300003E1040EDB5034DA95D90AE2050EDBCF30
:104A4000E7FF150EDB50E75E050EE7CFDBFF02D078
:104A5000050EDB6A040EDBCF2EF0160E45D9D8808A
:104A60002E5414E2160EDBCFE6FF150EDBCFE6FF69
:104A7000040EDBCFE6FF050EDB50E552E75CE552A6
:104A8000D880E754E552D880E7545FD9030EDB5055
:104A9000010B0BE1080EDB5008E0B2D801E08DD02D
:104AA000080EDB50BED8080EDB6A170EDB5007E09D
:104AB00088D9170EF1D903E12F1C01E17ED0160E23
:104AC000DB5016E07ED9300EE66E9FD802E12F1C37
:104AD00074E077D9DFCFE6FF42EC2CF0E552E552E7
:104AE000E552F4CF2FF00001F31C02E12F1C65E02A
:104AF000050EDBCF2EF0160EDB50D8802E5409E2C7
:104B0000050EDBCFE7FF160EDB50E75E050EE7CFA5
:104B1000DBFF300EE66E050ECBD94FE1390EDB2AF6
:104B2000DBCFE9FF3A0E01E3DB2ADBCFEAFF090E18
:104B3000EFCFDBFFDB500EE044D9090EADD902E127
:104B40002F1C3BE0390EDB2ADBCFE9FF3A0EEDE309
:104B5000DB2AEBD755D831E1160EDBCFE6FF080E86
:104B6000C3D8E552E7245DD82ED0070EDB50030AE8
:104B70001CE0010A14E0030A07E07BD9DBCFEEFF5B
:104B8000020EDBCFEDFF1FD0F5D8336A31AE02D075
:104B9000326833682CD8BCD833C0EEFF14D0EAD8C2
:104BA00031BE326824D8B4D80ED063D9DBCFEFFF42
:104BB0000AD07BD905E12F1C03E1F368F46810D01B
:104BC000FCD801E3DB2A79D982EF21F0010EDBCF9B
:104BD0002EF0020EDBCF2FF02EC0F3FF2FC0F4FF1C
:104BE0003B0EE15C02E2E16AE552E16ECBD029D9ED
:104BF000020EE8EF26F061D90800F550DF6E1200D2
:104C0000200EE66E080E58EF27F042EC2CF0E5522D
:104C1000E552E552F3CF2EF0F4CF2FF00001F31C54
:104C200012002E6E2F6AD950010F4DD92E50EE264C
:104C30002F50ED221200325E000E335AF70E32C0B2
:104C4000DBFFF80E33C0DBFF32C0E9FF33C0EAFF01
:104C50001200DBCFF4FFF350F45C1200DB50E76E80
:104C6000040EE7CFDBFF12000A0EDBCF2EF00B0E97
:104C7000DBCF2FF00C0EDBCF30F00D0EDBCF31F0A1
:104C80002E502F10301031101200130EEECFDBFF1C
:104C9000140EEDCFDBFF130EDBCF2EF0140EDBCFA7
:104CA0002FF00001800E2F141200F70EDBCF32F030
:104CB000F80EDBCF33F01200050EDB50E66ED95054
:104CC000130F01D9E552E750EE6EED6A12000A0E9D
:104CD000DBCF20F00B0EDBCF21F00C0EDBCF22F070
:104CE0000D0EDBCF23F01200DBCFE6FF150EDBCF7E
:104CF000E6FF050EDB50E552E724E552E7241200FB
:104D0000DB50CED8010EF36E060EF3CFDBFF1200A0
:104D1000EE50EFCFEAFFE96E30C0EEFF31C0EEFF9C
:104D200032C0EEFF1200D9CFE6FFDACFE6FFE1CFC7
:104D3000D9FFE2CFDAFF1200DFCFE6FFE66A11EC1F
:104D40002DF0E552E552F3501200E76E080EE7CF62
:104D5000DBFF1200EECF2EF0EECF2FF0EFCF30F0D2
:104D6000316A1200050EDBCF2EF0150EDB50D88015
:104D70002E541200010EDBCF30F0020EDBCF31F0EB
:104D8000326A1200E552E5CFDAFFE7CFD9FF120011
:104D90000A0E2EC0DBFF0B0E2FC0DBFF1200D95016
:104DA0000A0F63EF27F0F36E070EF3CFDBFF12005D
:104DB000EECF2EF0EFCF2FF01200010EDB2A020E05
:104DC0001200FC0EDBCFE6FFFD0EDBCFE6FF12008C
:104DD0002E5E000E2F5AF70E2EC0DBFFF80E2FC0EE
:104DE000DBFF2EC0E9FF2FC0EAFF1200DA20EA6ED7
:104DF000EF2AEECFF6FF000EEF22EECFF7FFEF2205
:104E0000EECFF8FF1200040EDBCFE6FF130EDB50EF
:104E1000E552E75C9ADFDB5004DF060EDB50120040
:104E2000090EDB500A0DF350DF24D00FE76E090E98
:104E3000E7CFDBFFFBEF25F0DB50F36E050E29EF2C
:104E400026F0F70EDBCF2EF0F80EDBCF2FF012009E
:104E5000DFCFE6FF05EF26F028DF030EECDEAAEF3A
:104E600026F057EC21F0E552E552E552E5520009F3
:104E70001200BDDEEE50EFCFEAFFE96E010E120028
:104E8000130EDB50F36E040E29EF26F0040EDB50F8
:104E9000F36E090E29EF26F0DBCFE6FF05EF26F0D3
:104EA000E76E050EE7CFDBFF12008BDF28EF27F060
:104EB000DBCFE6FF86DF31EF27F0D950F90FE96E3F
:104EC000FF0EF6EF26F0E96E000EDA20EA6E120011
:104ED000040140511F0B010801E012004051600B1A
:104EE000E842E842E842E842E842010801E01200F4
:104EF000445103E0440501E012004151220A31E02F
:104F0000030A24E0010A15E0210A0DE0010A01E08C
:104F100012000001E00E796F020E7A6F080E7C6FAE
:104F20007D6B7B8121D00001E00E796F020E7A6FDC
:104F30001BD046C481F047C482F00001880E7E6F0A
:104F4000050E7F6F836B846B808F12000001880ECB
:104F5000796F050E7A6F070E7C6F7D6BC10E7B6FCC
:104F6000120042C4DBF200017B8F12000501886B46
:104F70004B0E896F8A6B8B6B8C6B8D6B080E8E6FF3
:104F80000201CF6B1A0EE66E020EE66EC5EC1FF044
:104F9000E552E5521E0EE66E030EE66EC5EC1FF0FE
:104FA000E552E552400EE66E080EE66E050EE66E20
:104FB000E66A030EE66E6AEC20F02E6E050EE15EE8
:104FC0002E50F3CFD7F2F4CFD8F20201D96BDA6BBF
:104FD000D06B1200D9CFE6FFE1CFD9FF0201CF6B32
:104FE000D751D81102E1000E08D0D7C2E9FFD8C2CC
:104FF000EAFFEF50800B01E0010E000945E1FC0ED5
:10500000DBCF2EF0D7C2E9FFD8C2EAFFEE52EF5055
:10501000D8802E5408E2D7C2E9FFD8C2EAFFEE5288
:10502000FC0EEFCFDBFFCF6BFC0EDB50CF5D19E248
:10503000CF51EA6A080FE96E050EEA22EF50E66EDC
:10504000CF51E76EFD0EDBCFE9FFFE0EDBCFEAFFAF
:10505000E750E926000EEA22E552E750EF6ECF2B2B
:10506000E3D7400EE66E080EE66E050EE66EE66AC3
:10507000030EE66E6AEC20F02E6E050EE15E2E50F9
:10508000F3CFD7F2F4CFD8F20201CF51E552E7CFF8
:10509000D9FF1200D9CFE6FFE1CFD9FFA09A0201D4
:1050A000D0510CE1FD0EDBCFD1F2FE0EDBCFD2F200
:1050B000FC0EDBCFD5F2010ED66FD06FA08AE55281
:1050C000E7CFD9FF1200D9CFE6FFE1CFD9FF030E1A
:1050D000E126A09A0201D0512DE1DF6AFD0EDBCF5F
:1050E00022F0FE0EDBCF23F0DE5222C0DEFF23C013
:1050F000DDFFDD52DF2ADF502E6E2F6AFF0E2E18E5
:1051000002E12F500BE0010EDBCFE9FFDB2A020E9C
:10511000DBCFEAFF01E3DB2AEF50ECE1FD0EDBCF52
:10512000D1F2FE0EDBCFD2F2DFCFD5F20201010EBB
:10513000D66FD06FA08A030EE15C02E2E16AE5520D
:10514000E16EE552E7CFD9FF1200D9CFE6FFE1CFFC
:10515000D9FF030EE126A09A0201D0512EE1DF6AA9
:10516000FD0EDBCF22F0FE0EDBCF23F0DE5222C09D
:10517000DEFF23C0DDFFDD52DF2ADF502E6E2F6AF7
:10518000FF0E2E1802E12F500CE0010EDBCFF6FFD0
:10519000DB2A020EDBCFF7FF01E3DB2A0800F55024
:1051A000EBE1FD0EDBCFD1F2FE0EDBCFD2F2DFCF93
:1051B000D5F20201D66B010ED06FA08A030EE15C1E
:1051C00002E2E16AE552E16EE552E7CFD9FF120053
:1051D000D9CFE6FFE1CFD9FF020EE126A09A020166
:1051E000D951DA1102E1000E08D0D9C2E9FFDAC2C2
:1051F000EAFFEF50800B01E0010E000906E1030E0B
:10520000D05D01E1D06BD05102E1A08A7ED0020EC8
:10521000D05D16E1E66A000EE66EE66A010EE66E05
:10522000030EE66E6AEC20F02E6E050EE15E2E5047
:10523000F3CFD9F2F4CFDAF20201030ED06F64D0CB
:10524000D00562E1400E2E6E2F6AD5512E5C000E05
:105250002F5803E2400EDF6E02D0D5C2DFFFDF50D1
:10526000D55DD56F480ED36F050ED46F010EDFCF1D
:10527000DBFFD65116E1010EDB5028E0D1C2F6FF6C
:10528000D2C2F7FF0800F550D3C2E9FFD4C2EAFF4B
:10529000EF6ED32B000ED423D12BD223010EDB06CD
:1052A000EAD7010EDB5012E0D1C2E9FFD2C2EAFF19
:1052B000EF50D3C2E9FFD4C2EAFFEF6ED32B000E4A
:1052C000D423D12BD223010EDB06EBD70201D5511B
:1052D00007E1400EDF5C02E1020E01D0030ED06F49
:1052E000DFCFE6FF480EE66E050EE66E010EE66EB7
:1052F000030EE66E6AEC20F02E6E050EE15E2E5077
:10530000F3CFD9F2F4CFDAF2A08A020EE15C02E226
:0E531000E16AE552E16EE552E7CFD9FF1200E7
:02531E005374C6
:10532000617475733D25690D0A002135204572723F
:105330003A204E65656420636F6D6D61206E6578FF
:10534000742C20666F756E643A20272563270D0A3A
:105350000050492C2531750D0A004D522C25303353
:10536000750D0A002C25303475004100492C25307C
:1053700033692C253033692C253033692C253033A3
:10538000692C253033690D0A002138204572723AA4
:1053900020556E6B6E6F776E20636F6D6D616E64FE
:1053A0002027256325633A253258253258270D0AD0
:1053B000002138204572723A20556E6B6E6F776E01
:1053C00020636F6D6D616E64202725633A25325826
:1053D000270D0A002137204572723A2045787472F1
:1053E00061207061726D617465720D0A0021362052
:1053F0004572723A20496E76616C69642070617200
:10540000616D7465722076616C75650D0A002134DA
:10541000204572723A204D697373696E672070611E
:1054200072616D657465722873290D0A002133203D
:105430004572723A20525820427566666572206F36
:1054400076657272756E0D0A002132204572723ACD
:1054500020545820427566666572206F76657272B8
:10546000756E0D0A002130200D0A002008002573FA
:0D547000001B5B421B5B314B1B5B30470098
:02547E001A6AA8
:10548000E86A28AE4CEF2AF0256C261E271E281E3F
:105490002622272228221A1E23AE57EF2AF0206C3C
:1054A000211E221E231E2122222223221A1E23EC29
:1054B0002DF023BE6EEF2AF01AAE000C206C211ED8
:1054C000221E231EE86A2122222223221C6C1D1E7A
:1054D0001E1E1F1E1D221E221F22000C1ABE5EEF62
:1054E0002AF01B88FF0C23C02DF022C02CF021C015
:1054F0002BF021502602F4CF1FF0F3CF1EF02250E4
:105500002702F4CF21F0F3CF20F02602F3501F261C
:10551000F4502022E86A21222B502702F3501F2644
:10552000F4502022E86A212223502602F35020263C
:10553000F450212223502702226AE86A2222F350E3
:105540002126F45022222B502802F3502026F4501A
:105550002122236AE86A222223222C502802F350B7
:105560002126F4502222E86A23222D502802F350EB
:105570002226F4502322000C23C02DF022C02CF050
:1055800022502702F4CF21F0F3CF20F0235028023D
:10559000F4CF23F0F3CF22F02702F3502126F4506A
:1055A0002222E86A23222C502802F3502126F450AC
:1055B0002222E86A232228AEE2EF2AF02C50225E53
:1055C0002D50235A2DAE000C2750225E2850235A0E
:0255D000000CCD
:0E55D20008D80001605102E140EC21F0C8EC65
:1055E00006F0F8D70F0EC11202EC06F04FEF18F0DC
:1055F000120012001200120068EF27F01200B6EF3E
:1056000027F06D840101080EF56F070EF66FF507A0
:10561000000EF65BF551F611FAE16D941200D9CF48
:10562000E6FFE1CFD9FFFD0EDBCF22F0FE0EDBCF90
:1056300023F0720E221801E1235033E0E8682218AB
:1056400002E17F0E23182BE0740E221801E1235093
:1056500024E0750E221801E123501DE0730E22187C
:1056600001E1235016E0030E221801E123500FE060
:10567000020E221801E1235008E0010E221801E178
:10568000235001E010D0BBDF0FD0B8DF0DD0B4DF66
:105690000BD0B0DF09D0ACDF07D0ABDF05D0ABDF7C
:1056A00003D0000001D000D0010E00D0E552E7CFBA
:0456B000D9FF12000C
:0C56B4001E0EF66E080EF76E000EF86E6B
:1056C00001010900F550F06F0900F550F16F03E199
:1056D000F06701D03DD00900F550EB6F0900F5509F
:1056E000EC6F0900F550ED6F09000900F550E96E07
:1056F0000900F550EA6E090009000900F550EE6F47
:105700000900F550EF6F09000900F6CFF2F1F7CF6D
:10571000F3F1F8CFF4F1EBC1F6FFECC1F7FFEDC107
:10572000F8FF0101EE5302E1EF5307E00900F550E5
:10573000EE6EEE07F8E2EF07F9D7F2C1F6FFF3C11C
:10574000F7FFF4C1F8FF0101F007000EF15BBFD7CE
:02575000120045
:0E575200FE0EE3CFE9FFFF0EE3CFEAFFE9CF43
:10576000F3FFEACFF4FFFB0EE35003E1FC0EE3503E
:1057700009E0FB0EE30602E2FC0EE306FD0EE35039
:10578000EE6EF1D71200FE0EE3CFE9FFFF0EE3CF7E
:10579000EAFFF36AF46AEE5203E0F34AF42AFBD715
:1057A0001200FF0EE3CFF8FFE552FF0EE3CFF7FF45
:1057B000E552FF0EE3CFF6FFE552E66AE66AE66AD7
:1057C0000900F55209E0FD0EE32A05E1FE0EE32A89
:1057D00002E1FF0EE32AF4D7FD0EE3CF21F0FE0E27
:0C57E000E3CF22F0FF0EE3CF23F0120015
:0457EC00D9CFE6FF2C
:1057F000DACFE6FFE1CFD9FFE2CFDAFFE652E65299
:10580000E652E652D950FB0F2E6EFF0EDA202F6EB5
:105810002EC0DEFFDD6EDECFE6FFDDCFE6FFFB0E46
:10582000DBCFE6FFFC0EDBCFE6FFFD0EDBCFE6FFB6
:10583000F7C1E6FFF8C1E6FF6DEC21F02E6E070E12
:10584000E15C02E2E16AE552E16E2E50020EF3CF16
:10585000DBFF030EF4CFDBFF020EDBCF2EF0030ED7
:10586000DBCF2FF02EC0F3FF2FC0F4FF040EE15C5E
:1058700002E2E16AE552E16EE552E5CFDAFFE7CFF9
:04588000D9FF12003A
:0C588400D9CFE6FFDACFE6FFE1CFD9FF75
:10589000E2CFDAFFFB0EDBCF2EF0FC0EDBCF2FF0DA
:1058A0000001800E2F141AE1FB0EDBCFE9FFFC0E86
:1058B000DBCFEAFFEECFF3FFEDCFF4FFEE2A000ED1
:1058C000EF22F3CFE9FFF4CFEAFFFD0EDBCFEFFFCE
:1058D000EF502F6AF36E2FC0F4FF10D0FB0EDB5099
:1058E000FE0806E1FD0EDBCFE6FF76EC2DF005D0DD
:1058F000FD0EDBCFE6FFEEEC08F0E552E552E5CF1A
:08590000DAFFE7CFD9FF120026
:08590800120100020200004040
:10591000D80492FD82010102000109024300020144
:1059200000C0320904000001020201000524001039
:1059300001042402020524060001052401000107D8
:1059400005820308000209040100020A00000007A2
:10595000050302400000070583024000000403091C
:105960000418035300630068006D0061006C007A46
:10597000004800610075007300080355004200579D
:09598000001A595D596159795969
:06598A0020502502F3CFBE
:105990001CF0F4CF1DF02602F3501D26000EF4205B
:1059A0001E6E20502702F3501E26000EF4201F6E9C
:1059B00020502802F3501F2621502502F3501D26A7
:1059C000F4501E22000E1F2221502602F3501E26E4
:1059D000F4501F2221502702F3501F262250250287
:1059E000F3501E26F4501F2222502602F3501F2689
:0A59F00023502502F3501F26120079
:0659FA00FF0EE124E96E3E
:105A0000FF0EE220EA6EEDCFF4FFEFCFF3FFF46676
:105A100007D0600EF36404D07B0EF36001D0F39ADC
:105A20001200F36AF46AFF0EE124E96EFF0EE22031
:105A3000EA6EED6607D02F0EEF6404D03A0EEF60E9
:065A400001D0F32A120060
:0A5A46001F6A1E6A1D6A1C6A200E0A
:105A5000E76ED89020362136223623361C361D3686
:105A60001E361F3625501C5C26501D5827501E58C8
:105A700028501F5809E325501C5E26501D5A2750F8
:0E5A80001E5A28501F5A202AE72EE4D7120083
:025A8E004F4B7C
:105A90000D0A000D0A005542572046572044205653
:0F5AA000657273696F6E20312E342E380D0A0037
:105AB000000EF36E00EE00F0080E01D81200EA604E
:105AC00002D0EE6AFCD7F350E9601200EE6AFCD710
:105AD00016EE00F026EE00F0F86A1B9C5AEC2BF054
:0C5AE00003EC04F0E9EC2AF0FBD7120004
:045AEC00FF0EE35076
:105AF000ACBA04D0AF6AAB8EAC8A949CACA2FED791
:085B0000AD6EF36EF46A1200B1
:085B0800FF0EE350E84E12000D
:0E5B1000000000D000D000D0E82EFAD712001E
:025B1E00303124
:0F5B200032333435363738396162636465660075
:015B2F000075
:105B30000000000000000000000000000000000065
:105B40000000000000000000000000000000000055
:105B50000000000000000000000000000000000045
:105B60000000000000000000000000000000000035
:105B70000000000000000000000000000000000025
:015B80000024
:00000001FF
